:100000000C942A001895000018950000189500001F
:10001000189500001895000018950000189500002C
:10002000189500001895000018950000189500001C
:10003000189500001895000018950000189500000C
:1000400018950000189500001895000018950000FC
:10005000189500008FE58DBFC0E4E8E14E2E84E0E6
:100060008EBFD4E0F4E05F2EEEEFF3E0A0E6B0E068
:10007000A89584B7082E877F84BF88E1992781BD22
:1000800091BD88278D933197E9F766248FEF81BB67
:1000900001E40F930FE90F9300E20F931F911032C9
:1000A00039F41F911F3921F41F91113409F4FFCF46
:1000B000909AF894FFCF3197F1F70895689462F819
:0800C0000895E89462F8089528
:00000001FF
